:10000000830100308A00042883016D2F8207FF34AA
:10001000893489348934763400348434FD3484342A
:100020000034FF34803480348034803400348434AD
:10003000FD3484340034FF3402340C340234FF3491
:100040000034003400340034003438344034803418
:100050004034383400347034A834A834A834B03470
:100060000034003400340034003401340134FF34EF
:10007000013401340034FF348934893489348134C3
:100080000034FF3418342434423481340034FF34D3
:10009000043408341034FF3400348434FD348434A0
:0E00A0000034FF3418342434423481340034E8
:100EBE0083120313A0000430A1005330A200A20B32
:100ECE00662FA10B642FA00B622F080050308312E7
:100EDE000313A100831686018501073083129F003C
:100EEE008601A2012208273E840083138001A20AF4
:100EFE0010302202031C792FF230A300FF30A40021
:100F0E002108F000F1017108803AF2002408803ABD
:100F1E007202031D942F2308700283120313A20181
:100F2E00031C792F22082307A50024080318240A7E
:100F3E00A600A61FA72F2208273E84008313800138
:100F4E00A61BC72F2108F000F101FF30F007031C8C
:100F5E00F1077108803AF2002608803A7202031DEA
:100F6E00BA2F2508700283120313031CC92F2208FF
:100F7E00273E8400831300308A0025080620800057
:100F8E00831203132108F000F1017108803AF20078
:100F9E002608803A7202031DD62F25087002031808
:100FAE00DF2F2208273E8400831380018312031350
:100FBE00A20A10302202031C992FA001A2012208BE
:100FCE00273E8400831300088600220885004330E4
:100FDE00B700B70BF02FA20A10302202031CE62F27
:100FEE00A00A28302002031CE52FA30A0319A40A25
:020FFE00872F3B
:00000001FF
